:100000000C941E060C94CC270C94F9270C944606ED
:100010000C9446060C9446060C9446060C94460630
:100020000C9446060C9446060C94E2120C94460678
:100030000C9446060C9446060C9446060C94460610
:100040000C9426280C9446060C94142C0C94572CD3
:100050000C9446060C9446060C9446060C944606F0
:100060000C9446060C9446064618A81887188A1859
:100070008D189018931896189918A818A218DA19BC
:10008000DC19DC19DA19DC19DC19DC19DC19DC19CA
:10009000DC19DC19DC19DC19DC19DC19DC19DC19B8
:1000A0006019DC19DC19DC19DC19DC19D118DC1930
:1000B000DC19DC19DC19DC19DC19DC19DC19DC1998
:1000C000DC19DC19DC19DC19DC19DC196C196C1968
:1000D0006C196C196C196C196C196C196C19DC1988
:1000E000DC19DC19DC19DC19DC19D1186B196B1956
:1000F0006B196B19DC1979197F1985198B199119ED
:1001000097199D19A319AD19B719C119CB1912194E
:10011000D418DC19DC19DC19DC196019DC19DC19BC
:10012000DC19DC19DC19DC19DC19DC196A196A190B
:100130006A196A19DC1979197F1985198B199119AE
:1001400097199D19A319AD19B719C119CB1912190E
:10015000D418DC19DC19DC19DC1960190F1A0F1A14
:100160000F1A0F1A0F1A0F1A0F1A0F1A0F1A0F1A47
:100170000F1A0F1A0F1A261B261B261B261B261BBF
:10018000261B541A5E1A681A721AD01ADA1AE91A59
:10019000FA1A821C971CA31CAC1CBB1CE01CE91C9B
:1001A000321DFB1C45204B20512058206620882002
:1001B000A620456E746572206D656E752E2E2E001C
:1001C000546F67676C6564206D6963726F50504D42
:1001D00000546F67676C656420696E76657274653C
:1001E000642050504D2100546F67676C6564205443
:1001F00058206D7574696E672100546F67676C6570
:10020000642074656C656D65747279210050726F3D
:10021000746F636F6C206572726F72207769746897
:100220002052580054696D656F7574207768656E4B
:1002300020636F6E6E656374696E6720746F205201
:100240005800507265737320616E79206B65792058
:10025000746F2063616E63656C00436F6E6E6563DF
:1002600074696E6720746F2052582C20706F776508
:100270007220757020746865205258202877697440
:10028000682062696E6420706C7567206966206EF4
:100290006F74207573696E6720616C776179732064
:1002A00062696E642900546F67676C656420276912
:1002B0006D6D656469617465206F75747075742700
:1002C00000546F67676C65642027736C61766520E6
:1002D0006D6F64652700546F67676C6564202761E4
:1002E0006C776179732062696E642700546F676769
:1002F0006C65642050504D206368616E6E656C20A3
:100300006C696D69740053657420525353492069B8
:100310006E6A656374696F6E206368616E6E656C8A
:100320002028303D3D64697361626C652900536526
:10033000742050504D206D696E696D756D20737914
:100340006E630053657420626561636F6E20696E31
:1003500074657276616C0053657420626561636FC9
:100360006E2064656C617900536574206265616319
:100370006F6E206672657175656E637920696E2097
:10038000487A3A20303D64697361626C652C205074
:10039000783D504D52206368616E6E656C20782CFC
:1003A0002046783D465253206368616E6E656C202E
:1003B00078005365742050574D2073746F7020641B
:1003C000656C61792028302064697361626C6564B2
:1003D0002C20312D323535203D3D20302E317320FB
:1003E0002D2035306D696E29005365742050504DB5
:1003F0002073746F702064656C61792028302064EC
:10040000697361626C65642C20312D323535203D75
:100410003D20302E3173202D2035306D696E29003E
:10042000536574206661696C736166652064656CF0
:1004300061792028302064697361626C65642C20C6
:10044000312D323535203D3D20302E3173202D2089
:1004500035306D696E29002A2A2A2A2A2A2A2A2A50
:100460002A2A2A2A2A2A2A2A2A2A2A2A2A2A2A2AEC
:100470002A2A2A2A0052582041636B6564202D20C5
:1004800072657665727420737563636573736675E0
:100490006C21002A2A2A2A2A2A2A2A2A2A2A2A2AAD
:1004A0002A2A2A2A2A2A2A2A2A2A2A2A2A2A2A2AAC
:1004B000002A2A2A2A2A2A2A2A2A2A2A2A2A2A2AC6
:1004C0002A2A2A2A2A2A2A2A2A2A2A2A2A2A00528E
:1004D000582041636B6564202D20757064617465DC
:1004E000207375636365737366756C21002A2A2A0D
:1004F0002A2A2A2A2A2A2A2A2A2A2A2A2A2A2A2A5C
:100500002A2A2A2A2A2A2A2A2A2A0056616C696457
:100510002063686F69636573206172653A205B319F
:100520005D2D5B31365D20286368616E6E656C20E1
:10053000312D31362900536574206F7574707574D0
:1005400020666F7220706F727420005B585D2061AE
:10055000626F7274206368616E67657320616E6498
:10056000206578697420525820636F6E6669670051
:100570005B535D20736176652073657474696E6783
:100580007320746F205258005B525D20726576654F
:1005900072742052582073657474696E6773207486
:1005A0006F2064656661756C747300557365206EA9
:1005B000756D62657273205B312D445D20746F2010
:1005C0006564697420706F727473205B452D515D92
:1005D00020666F722073657474696E677300202DD6
:1005E00020726563656976657220636F6E66696700
:1005F000757261746F722C20727820737720000AF4
:100600000A6F70656E4C52536E67200053657420FC
:1006100073657269616C2062617564726174653AB8
:10062000200056616C69642063686F696365733A82
:100630002031202D20342B34202F2032202D203823
:10064000202F2033202D20382B34202F2034202D14
:10065000203132202F2035202D2031322B34202FF5
:100660002036202D20313600536574204368616E9A
:100670006E656C20636F6E6669673A20005365741F
:100680002044617461726174652028302D32293AEA
:10069000200053657420486F70206368616E6E653A
:1006A0006C7320286D61782032342C207365706162
:1006B000726174656420627920636F6D6D61732966
:1006C0002076616C69642076616C75657320312DCC
:1006D0003235353A2000536574206368616E6E656B
:1006E0006C2073706163696E6720287831306B48C5
:1006F0007A293A200053657420524620706F77653E
:10070000722028302D37293A200053657420524634
:10071000206D6167696320286865782920652E67E8
:100720002E20307844454144463030443A2000532E
:1007300065742062617365206672657175656E63AC
:10074000792028696E20487A293A20005B5A5D207A
:10075000656E746572207265636569766572206383
:100760006F6E66696775726174696F6E2075746902
:100770006C79005B465D20646973706C61792061FF
:10078000637475616C206672657175656E63696509
:10079000732075736564005B525D2063616C6375E3
:1007A0006C6174652072616E646F6D206B65792079
:1007B000616E6420686F70206C697374005B495DC2
:1007C000207265696E697469616C697A6520736508
:1007D0007474696E677320746F20736B65746368DB
:1007E0002064656661756C7473005B585D2072658A
:1007F00076657274206368616E67657320616E64EC
:100800002065786974206D656E75005B535D20739B
:100810006176652073657474696E677320746F20E8
:10082000454550524F4D20616E64206578697420B3
:100830006D656E7500557365206E756D62657273BA
:10084000205B302D395D20746F20656469742070E1
:100850006172616D657465727300202D2053797328
:1008600074656D20636F6E66696775726174696F18
:100870006E000A0A6F70656E4C52536E672000510D
:1008800029204F7574707574206265666F726520DB
:100890006C696E6B20283D465329203A2000502970
:1008A00020536C617665206D6F64652028657870D3
:1008B0006572696D656E74616C293A20004F29205C
:1008C00054696D65642042494E44206174207374FC
:1008D000617274757020203A20004E292050504DCE
:1008E000206F7574707574206C696D69746564200F
:1008F000202020203A200044495341424C454400E6
:100900004D292050504D205253534920746F20637D
:1009100068616E6E656C202020203A20004C2920F2
:1009200050504D206D696E696D756D2073796E63E1
:10093000202875732920203A200044495341424C15
:100940004544004B29204661696C736166652062ED
:100950006561636F6E20696E74762E2028312D32AA
:10096000353573293A20004A29204661696C736144
:10097000666520626561636F6E2064656C617920D5
:1009800028302D323535203D3E20313073202D204A
:100990003135306D696E293A200049292046616958
:1009A0006C7361666520626561636F6E206672714B
:1009B0002E203A200048292050574D2073746F7024
:1009C0002064656C6179202020202020203A2000BE
:1009D00047292050504D2073746F702064656C61FE
:1009E00079202020202020203A200046292046611E
:1009F000696C736166652064656C617920202020D4
:100A00002020203A200050574D206368616E6E65AB
:100A10006C200066756E6374696F6E3A2000292041
:100A2000706F72742000506F776572546F776572C3
:100A300000445446205548462033322D62697420C4
:100A400031306368004F70656E4C52536E67525878
:100A5000206D696E6920342F36636800466C7974A6
:100A6000726F6E2F4F72616E6765525820554846FF
:100A70002038636800525820747970653A20004429
:100A8000697361626C656400487A00203D3D200016
:100A900043616C63756C61746564207061636B6540
:100AA0007420696E74657276616C3A200042292068
:100AB0004D6963726F202868616C66292050504D23
:100AC000202020203A00412920496E766572746505
:100AD000642050504D20696E20202020203A0030A4
:100AE00029204D7574652062757A7A657220286DAB
:100AF0006F73746C79293A003929205365726961E2
:100B00006C2062617564726174653A00736D617224
:100B100074506F7274004672536B79005472616E38
:100B200073706172656E740044697361626C6564B0
:100B30000038292054656C656D657472793A2020FF
:100B40002020202020003729204368616E6E656CCC
:100B500020636F6E6669673A202000362920446161
:100B60007461726174652028302D32293A2020206A
:100B700000352920486F70206368616E6E656C7364
:100B80003A2020202020003429204368616E6E65C1
:100B90006C2073706163696E673A202000332920EE
:100BA000524620706F7765722028302D37293A2001
:100BB0002020003229205246206D616769633A2067
:100BC0002020202020202020003129204261736530
:100BD000206672657175656E63793A202020000089
:100BE00000000700020100000304060000000000EE
:100BF00000000001020408102040800102040810D7
:100C00002001020408102004040404040404040263
:100C10000202020202030303030303000000002395
:100C2000002600290000000000250028002B0000FD
:100C3000000000240027002A0000452D11241FBEBB
:100C4000CFEFD8E0DEBFCDBF13E0A0E0B1E0E8E930
:100C5000F0E602C005900D92A83CB107D9F716E066
:100C6000A8ECB3E001C01D92AE38B107E1F71CE07B
:100C7000CCE3DCE004C02297FE010E944E2ECA3372
:100C8000D107C9F70E94812D0C944A300C940000C2
:100C900080917305813019F482E08093730580910F
:100CA0007305833019F484E0809373050895A89543
:100CB0000895DC01ED91FC910190F081E02D099502
:100CC00008952091740530917505382748E0C901D1
:100CD000880F991F37FF06C09C0151E2252750E17C
:100CE000352701C09C01415091F730937505209341
:100CF0007405089588E38093760580E092ECA1E086
:100D0000B0E08093770590937805A0937905B09330
:100D10007A0587E08093830580EC9AECA9E8B6E336
:100D200080937B0590937C05A0937D05B0937E0511
:100D300085E0809384058DEE9EEFADEABEED809355
:100D40007F0590938005A0938105B0938205E5E827
:100D5000F5E080E090E0863028F4DC01AE54BC4F32
:100D60002C9101C020E0219301968831910599F7DB
:100D700082E080939D058AE080939E05089580EC33
:100D800097EFAAEBB7E38093BB059093BC05A093C4
:100D9000BD05B093BE0580E090E0A0E0B0E5809393
:100DA000BF059093C005A093C105B093C205E3ECC5
:100DB000F5E080E081938F5F8031E1F70895A0E056
:100DC000B0E0E5EEF6E00C94172ED82F0E947C28B8
:100DD0006115710581059105C9F30E94BA2E109223
:100DE0007F05109280051092810510928205C4E063
:100DF000812C912C54018A94C0907F05D09080055D
:100E0000E0908105F0908205FE2CED2CDC2CCC24AA
:100E10000E94B52EA50194010E94F62D6C0D7D1D3A
:100E20008E1D9F1D60937F057093800580938105C3
:100E300090938205C15001F7DD2309F450C005E805
:100E400015E0E801A12CB12C62E3C62ED12CE12CD7
:100E5000F12C8881882309F442C0B39419F40E94CC
:100E60007A063DC00E94B52EA70196010E94F62D7C
:100E7000E1E0E60FA5E8B5E08A2F801B8A1520F493
:100E80008D918E13F9CFE9CF2091840530E0A0E158
:100E9000B7E20E948E2D9B01AC01AE2FB0E00E9404
:100EA0009D2D40907B0550907C0560907D05709055
:100EB0007E05640D751D861D971D4090BB055090E5
:100EC000BC056090BD057090BE05461657066806C5
:100ED000790618F2E993A39488E1A812BACFCDB7A6
:100EE000DEB7E0E10C94332E8436910520F4BC018A
:100EF00080E090E017C09C018E3B910528F42A55B4
:100F00003109AAE0B0E00CC0823D910528F4245BD1
:100F10003109A4E6B0E004C02D5C3109A8E5B2E0D7
:100F20000E948E2DA4E6B0E09B01AC010E949D2D95
:100F3000089590E08C599F4F0E947407089561E0D6
:100F40008AE00E94292960E08AE00E9462290895CF
:100F5000892B11F061E001C060E08AE00E94622903
:100F6000089560E08CE00E94292961E08BE00E94F6
:100F7000292961E08DE00E94292960E082E00E9439
:100F8000292961E084E00E942929089542E050E087
:100F900068E476E080E00E94AC270895E3E0F0E0AA
:100FA00089E080935700E491E67081E0E63009F033
:100FB00080E00895CF93DF93C82F0E94CE07882347
:100FC00081F0DFB781E080937205F8940E945706A4
:100FD00088E180936000C0936000C1110E945706B1
:100FE000DFBFDF91CF9108958F929F92AF92BF9212
:100FF000CF92DF92EF92FF92CF93FC01C0A5EC2F2E
:10100000E770F0E0E658FC4FA081B0E0C7FF03C0F6
:1010100024E130E002C02FE030E0FC0197A183E141
:10102000989FF0011124E25CFE4F80809180A280A5
:10103000B380A20FB31F20E43FE14DE750E00E94D0
:10104000A82DA50194010E94D42D8C2F887149F4FC
:1010500069017A01E0EDCE0EE7E0DE1EE11CF11C35
:101060001BC0C7FF05C060E47AE88CE29EE004C0C4
:1010700060E07EEE8AEB9BE069017A01F8EBCF0E2F
:10108000FBE0DF1EE11CF11CA50194010E94D42DA0
:10109000C20ED31EE41EF51EC701B60169517C4F76
:1010A0008F4F9F4F28EE33E040E050E00E94D42D58
:1010B000A8EEB3E00E949D2DCF91FF90EF90DF90BE
:1010C000CF90BF90AF909F908F9008958F3F9105E4
:1010D00051F048F0811522E0920738F081159340D5
:1010E00030F482E0089580E0089581E0089583E07F
:1010F0000895A0E0B0E0EFE7F8E00C94202EEB01BB
:101100008A01B82FB695A0E028813981F8012083A3
:101110002A813B8121832C813D8122832E813F8145
:101120002383688179814A815B812C813D81EE81B5
:10113000FF819F2F9295990F990F907C272F2370F5
:10114000922B252F2370220F220F922B232F2370F7
:101150002295207F922BF80194830B5F1F4F2896D6
:10116000AF5FBA1788F680FF24C0888199810E94FA
:101170006608D82E8A819B810E946608E82E8C81A1
:101180009D810E946608F82E8E819F810E946608CC
:10119000F0E4DF9EA001112490E1E99E900111246A
:1011A000242B282BE4E0FE9EB0011124262BF8010D
:1011B0002083CDB7DEB7E7E00C943C2E803223E0ED
:1011C000920708F1883E23E0920740F48F51934044
:1011D000E4E096958795EA95E1F70895803D27E04C
:1011E000920718F48C5D93400895883928E092079F
:1011F00068F4885C974074E0969587957A95E1F756
:101200008D509C4F089580E090E008958FEF93E01B
:1012100008958C30910540F4A4E0880F991FAA9599
:10122000E1F7885D9C4F0895843F23E0920718F40E
:1012300084529C4F0895811524E0920740F486570C
:10124000934FF4E0880F991FFA95E1F7089580E92C
:1012500098E008959C013695279525753575821B74
:10126000930B9C0123733373969587959695879579
:1012700083739373820F931F9C0154E036952795D7
:101280005A95E1F7280F391F2F703F7041E051E068
:10129000249FC001259F900D349F900D1124892F0C
:1012A00008952D98882319F000002B9A02C00000A1
:1012B0002B9800002D9A000008952D9A000083B10C
:1012C0002D980000829581700895CF93DF93D82FD9
:1012D0005C9A2D985C98C8E08D2F80780E94510907
:1012E000DD0FC150C9F72D98DF91CF9108958F7709
:1012F0000E9465090895CF93DF93D82FC8E08D2F02
:1013000080780E945109DD0FC150C9F72D98DF91F7
:10131000CF910895CF93DF932D98C8E080E0D82F28
:10132000DD0F0E945D098D0FC150C9F7DF91CF918C
:1013300008950E9477090E948A095C9A0895A1E0A5
:10134000B0E0E5EAF9E00C94252E806869830E94FC
:1013500065096981862F0E947B095C9A2196E2E0EB
:101360000C94412ECF93C0917F05C827E82FF0E061
:10137000EA58FA4F678589E70E949F096C2F8DE331
:101380000E949F096C2F82E40E949F09CF910895CB
:1013900086E20E9499090895CF93DF93EC016C8156
:1013A0008CE10E949F096D818DE10E949F096E81F1
:1013B0008EE10E949F096F8180E20E949F096885EB
:1013C00081E20E949F09698582E20E949F096A85E5
:1013D00083E20E949F096B8584E20E949F096C85CD
:1013E00085E20E949F096D858AE20E949F096E85B1
:1013F0008EE60E949F096F858FE60E949F0968898B
:1014000080E70E949F09698981E70E949F096A8994
:1014100082E70E949F09DF91CF910895CF92DF92DA
:10142000EF92FF92CF93DF936B017C01C11488E3AD
:10143000D8068CE9E8068CE1F80628F5C701B60164
:1014400020E836E948E950E00E94D42DE901689788
:1014500060E879E687E69FEF0E94B02D6C0D7D1D58
:101460008E1D9F1DF2E0660F771F881F991FFA954A
:10147000D1F721E732E040E050E00E94D42DF22E77
:10148000E32E80E421C0C701B60120E03DE241E344
:1014900051E00E94D42DE901689760E073ED8EEC75
:1014A0009EEF0E94B02D6C0D7D1D8E1D9F1D660F41
:1014B000771F881F991F21E732E040E050E00E942B
:1014C000D42DF22EE32E80E66C2F6F71680F85E726
:1014D0000E949F096E2D86E70E949F096F2D87E766
:1014E0000E949F09DF91CF91FF90EF90DF90CF9006
:1014F0000895682F8DE60E949F0908958F929F920C
:10150000AF92BF92CF92DF92EF92FF92CF93DF9391
:10151000D82F83E00E9499098093710584E00E948E
:1015200099098093700560E086E00E949F0961E060
:1015300087E00E949F096FE789E00E949F0965E0AC
:101540008AE00E949F0962E18BE00E949F0965E1A9
:101550008CE00E949F096DEF8DE00E949F0960E082
:101560008EE00E949F09DD2319F08BE291E008C014
:1015700020919D0533E1239FC0011124825C9E4F81
:101580000E94CC096CE880E30E949F096FE082E32F
:101590000E949F0962E483E30E949F0980919E0557
:1015A00087FF02C064E101C06AE084E30E949F09F2
:1015B0006AE285E30E949F096DE286E30E949F092B
:1015C00064ED87E30E949F0960E088E30E949F0921
:1015D00060E089E30E949F09D11109C0C0907F0596
:1015E000D0908005E0908105F090820507C0C5E9A4
:1015F000CC2EC1ECDC2EED2CCEEDFC2ECAE38F2CD4
:101600009924AA24BB24682D8C2F0E949F09682D41
:1016100085E08C0F0E949F09FE2CED2CDC2CCC2445
:10162000CF5FCE3361F76FEF83E40E949F096FEFC6
:1016300084E40E949F096FEF85E40E949F096FEF89
:1016400086E40E949F09DD2311F066E002C06091EC
:1016500083058DE60E949F0960E089E70E949F094B
:10166000609184058AE70E949F0960E083E70E94F9
:101670009F0960E084E70E949F09D11109C0609131
:101680007B0570917C0580917D0590917E0504C05D
:1016900060EC7AEC89E896E30E940E0ADF91CF9124
:1016A000FF90EF90DF90CF90BF90AF909F908F9082
:1016B000089561E087E00E949F0964E28EE70E943E
:1016C0009F0963E088E00E949F0960E088E00E9433
:1016D0009F0965E087E00E949F0962E085E00E9423
:1016E0009F0983E00E9499098093710584E00E941C
:1016F000990980937005089583E00E949909809369
:10170000710584E00E9499098093700561E087E08B
:101710000E949F096AE070E080E090E00E949F28AC
:101720000E94590B00000895CF92DF92FF920F9311
:101730001F93CF93DF931F92CDB7DEB7082F162FDD
:101740008EE399830E949F09F02EC02E9981D92E95
:101750008C2D8F19811738F4F60161916F018FE795
:101760000E949F09F5CF64E085E00E949F0983E015
:101770000E9499098093710584E00E9499098093E1
:1017800070050E947C2860936C0570936D058093B2
:101790006E0590936F0569E087E00E949F0981E0E4
:1017A000809373050F90DF91CF911F910F91FF9060
:1017B000DF90CF9008950F931F930E94940B809118
:1017C0007305813099F40E947C2800916C0510917A
:1017D0006D0520916E0530916F05601B710B820BBA
:1017E000930B603A76488140910548F380917305E8
:1017F000813031F46EE971E082EE95E00E94682A52
:101800001F910F9108950F931F938091730582305C
:1018100021F41092730581E020C08091730581301E
:10182000D9F40E947C2800916C0510916D052091DF
:101830006E0530916F05601B710B820B930B613A43
:1018400076488140910540F061E087E00E949F0961
:101850001092730582E001C080E01F910F910895FE
:10186000CF93DF93EC014AE050E06D2F70E082EE01
:1018700095E00E94362B6EE282EE95E00E943A2AB5
:10188000BE0184E0769567958A95E1F76F707727BA
:101890004AE050E082EE95E00E94362BDF91CF9136
:1018A0000895D82FC0E0CD1790F45E9A409A64E670
:1018B00070E080E090E00E949F285E98409864E687
:1018C00070E080E090E00E949F28CF5FECCF6CE258
:1018D00071E080E090E00E949F28E4CF0F931F9377
:1018E000CF93DF93EC01062F15E0115051F0CE019C
:1018F0000E943130081741F0602FCE010E9439302C
:10190000F4CF82E00E94510CDF91CF911F910F9193
:101910000895A0E0B0E0EFE8FCE00C94172E482E0C
:10192000562EC0E0D0E0612C712CE12CF12C00E0AF
:1019300010E041100CC06090D40586E4689E300130
:10194000112459E1E52EF12C0AEB15E01EC091E0BF
:1019500049120FC06090D405E6E46E9E3001112458
:10196000FBE16F0E711C49E2E42EF12C06E715E055
:101970000CC082E0481209C028E1622E77247394DB
:10198000EE24E394F12C03ED15E043018C0E9D1E33
:1019900010927505109274053401A62CA818B12C6C
:1019A000C30101966C01AE14BF04A8F4A00EB11ED1
:1019B000511006C0C3010E943130F501808305C07B
:1019C000F5016081C3010E946E0CF50180810E94C7
:1019D00061063601E2CFC301511018C0C3010E9455
:1019E0003130B82EC6010E9431302B2D30E0322F1D
:1019F0002227282B809174059091750582179307F3
:101A000079F4C0E0D0E05524539493CF360160912F
:101A100075050E946E0C60917405C6010E946E0CE3
:101A2000C05EDE4FC13E92E0D90708F482CF852D1B
:101A3000CDB7DEB7E0E10C94332E61E082E00E9486
:101A4000890C089560E082E00E94890C8091D305A2
:101A5000853028F084E08093D3050E941D0D80918D
:101A6000D3058093D405089561E080E00E94890C3D
:101A700061E081E00E94890C089560E080E00E94AE
:101A8000890C882351F060E081E00E94890C882352
:101A900021F080917605883349F00E94BF060E94AC
:101AA0007A0681E00E94DF060E94340D08958823A3
:101AB00019F06AEA71E002C06EEA71E082EE95E028
:101AC0000E94682A0895FF920F931F93CF93DF938C
:101AD00069EC7BE082EE95E00E94142A40917B0540
:101AE00050917C0560917D0570917E052AE030E083
:101AF00082EE95E00E943D2B63EB7BE082EE95E069
:101B00000E94142A40917F055091800560918105C3
:101B10007091820520E130E082EE95E00E943D2B3D
:101B20006DE97BE082EE95E00E94142A4AE050E0E5
:101B30006091830582EE95E00E94652B67E87BE06B
:101B400082EE95E00E94142A4AE050E060918405FC
:101B500082EE95E00E94652B61E77BE082EE95E0E6
:101B60000E94142AC5E8D5E0F12C8E0188818823D3
:101B7000A9F0FF2031F061EB71E082EE95E00E9468
:101B8000372A21964AE050E0F801608182EE95E024
:101B90000E942E2BF394F8E1FF12E7CF82EE95E03E
:101BA0000E94422A6BE57BE082EE95E00E94142AB7
:101BB0004AE050E060919D0582EE95E00E94652B21
:101BC00066E47BE082EE95E00E94142AE0919E0597
:101BD000E770F0E0EE0FFF1FEE57FC4F6081718160
:101BE00082EE95E00E94682A61E37BE082EE95E058
:101BF0000E94142A80919E058871883069F028F42B
:101C0000811113C068E27BE00CC0803141F0883163
:101C100061F46CE07BE005C06CE17BE002C066E152
:101C20007BE082EE95E00E94562A68EF7AE082EE31
:101C300095E00E94142A40917705509178056091B3
:101C4000790570917A052AE030E082EE95E00E94F5
:101C50003D2B6FED7AE082EE95E00E94142A809190
:101C6000BF0580710E94570D66EC7AE082EE95E028
:101C70000E94142A8091BF0580740E94570D6DEA5E
:101C80007AE082EE95E00E94142A8091BF0580726E
:101C90000E94570D60E97AE082EE95E00E94142AD6
:101CA00086E795E00E94F407AB01BC012AE030E032
:101CB00082EE95E00E941F2B6BE87AE082EE95E0C1
:101CC0000E94142A86E795E00E94F4079B01AC016C
:101CD00060E472E48FE090E00E94D42DBA01A90183
:101CE0002AE030E082EE95E00E941F2B68E87AE05F
:101CF00082EE95E00E94562ACDB7DEB7E5E00C945F
:101D00003E2E8F929F92AF92BF92CF92DF92EF9230
:101D1000FF92811107C06FE77AE082EE95E00E94A2
:101D2000562A2FC090E00E94740724E630E040E07D
:101D300050E00E94D42DCA01B9012AE030E040E011
:101D400050E00E94D42D49015A016B017C012AE028
:101D500030E0B501A40182EE95E00E941F2B6EE2F7
:101D600082EE95E00E943A2A2AE030E0B701A6010F
:101D700082EE95E00E941F2B63E782EE95E00E94C1
:101D80007A2AFF90EF90DF90CF90BF90AF909F9016
:101D90008F9008951F93CF93DF9365E77AE082EEEB
:101DA00095E00E94142A80919F05813041F46CE5F2
:101DB0007AE082EE95E00E94562A10E050C0823010
:101DC00019F465E47AE0F5CF843019F461E37AE040
:101DD000F0CF853091F766E27AE0EBCFC12FD0E00B
:101DE000C930D1050CF441C068E3610F82EE95E083
:101DF0000E943A2A6EE17AE082EE95E00E94142A6F
:101E0000BE016F5F7F4F4AE050E082EE95E00E9496
:101E1000FE2A63E17AE082EE95E00E94142AC15620
:101E2000DA4FE981E03218F566E07AE082EE95E07B
:101E30000E94142A8981803130F06DE673E082EED1
:101E400095E00E94372A69816F7070E06F5F7F4F65
:101E50004AE050E082EE95E00E94072B1F5F8091E0
:101E60004805181708F4BACF0FC061E3BECFEF7072
:101E7000F0E0EE0FFF1FEE56FC4F6081718182EEA5
:101E800095E00E94682AEACF6BEE79E082EE95E059
:101E90000E94142A8091B7050E94810E60ED79E0BE
:101EA00082EE95E00E94142A8091B8050E94810E6E
:101EB00065EB79E082EE95E00E94142A8091B905E5
:101EC0000E94810E6AE979E082EE95E00E94142A70
:101ED0004091AF055091B0056091B1057091B20588
:101EE000411551056105710539F12AE030E082EEB6
:101EF00095E00E943D2B67E679E082EE95E00E9436
:101F0000142A8091B3050E949907AB01BC012AE015
:101F100030E082EE95E00E943D2B63E479E082EEB2
:101F200095E00E94142A4AE050E06091B40582EEE8
:101F300095E00E94652B06C06AE379E082EE95E0A9
:101F40000E94562A6DE179E082EE95E00E94142A03
:101F50006091B5057091B6054AE050E082EE95E0DB
:101F60000E944F2B60E079E082EE95E00E94142AF7
:101F70006091AE05603450F470E06F5F7F4F4AE0CF
:101F800050E082EE95E00E94072B06C067EF78E0F4
:101F900082EE95E00E94562A6AED78E082EE95E0A6
:101FA0000E94142A8091AD0580FF03C063EB71E0AD
:101FB00002C067EB71E082EE95E00E94682A6DEB4B
:101FC00078E082EE95E00E94142A8091AD0582703F
:101FD0000E94570D6EE978E082EE95E00E94142A87
:101FE0008091AD0584700E94570D6FE778E082EE16
:101FF00095E00E94142A8091AD0588700E94570DCB
:10200000DF91CF911F9108950F931F93CF93DF938B
:10201000209145052F3FA9F56FEF75E082EE95E021
:102020000E94142A80E893E00E94300C6EED75E067
:1020300082EE95E00E94142A809146059091470512
:102040000E94300C6BEA75E082EE95E00E94562A01
:1020500068E875E082EE95E00E94562A60E775E038
:1020600082EE95E00E94562A6BE475E082EE95E0E0
:102070000E94562A82EE95E00E94422A0E94CA0ED1
:1020800068C012160CF065C0332727FD309580918B
:10209000480590E0821793070CF45BC066E375E097
:1020A00082EE95E00E94142A60914505772767FD2E
:1020B00070954AE050E082EE95E00E94072B6BE0BD
:1020C00075E082EE95E00E94142A10E008E280910B
:1020D00049051817D0F5C12FD0E0CC0FDD1FC65B26
:1020E000DA4F288130E080914505992787FD90954A
:1020F00001972817390739F56BEB71E082EE95E00F
:102100000E94372A4AE050E0602F82EE95E00E945C
:102110002E2B6FEB71E082EE95E00E94372AE98169
:10212000EF70F0E0EE0FFF1FEE56FC4F6081718103
:1021300082EE95E00E94372A63EC71E082EE95E032
:102140000E94372A0F5F1F5FC2CF82EE95E00E9488
:10215000422ADF91CF911F910F910895FF920F9323
:102160001F93CF93DF93C5E8D5E0F12C8E018881D2
:102170008823D1F165EC71E082EE95E00E94372A68
:102180004AE050E06F2D82EE95E00E942E2B62ED2A
:1021900071E082EE95E00E94372A2196F8012081B5
:1021A00030E0A0E1B7E20E948E2D9B01AC01A0912E
:1021B0008405B0E00E949D2DAB01BC0180917B05A0
:1021C00090917C05A0917D05B0917E05480F591F27
:1021D0006A1F7B1F2AE030E082EE95E00E943D2BD3
:1021E000F394F8E1FF12C2CFCDB7DEB7E5E00C946F
:1021F0003E2E1092DF0485E6E0EEF4E0DF011D9252
:102200008A95E9F70895CF93C82F8F3719F0883052
:1022100009F045C0E091DF04EE23D9F1E150E093ED
:10222000DF04F0E0E052FB4F10826DE070E082EEE0
:1022300095E00E945906C0E08091DF04C81760F461
:10224000EC2FF0E0E052FB4F608170E082EE95E011
:102250000E945906CF5FF0CF60E270E082EE95E019
:102260000E9459066DE070E082EE95E00E945906EA
:10227000C0E08091DF04C81778F5EC2FF0E0E05261
:10228000FB4F608170E082EE95E00E945906CF5FBF
:10229000F0CF67E082EE95E00E943A2A1DC08B31B4
:1022A00019F40E94F9101AC08D30C1F08A30B1F0D3
:1022B0008091DF04843668F76C2F70E082EE95E041
:1022C0000E945906E091DF0481E08E0F8093DF04C5
:1022D000F0E0E052FB4FC08380E001C081E0CF918D
:1022E0000895CF93C82F0E947C286093C8047093F0
:1022F000C9048093CA049093CB04C093DD04CC231B
:1023000029F040E051EE60E070E004C040E855E2A2
:1023100060E070E082EE95E00E94C42CCF910895B9
:102320009091CC04492F4F7050E0BA016F5F7F4FFE
:10233000292F30E0E4E035952795EA95E1F762171B
:10234000730759F0FA01E353FB4F808381E0890F53
:102350008F70907F892B8093CC0408956EE770E096
:1023600082EE95E00E9459060895A3E1B1E0EBEBFF
:10237000F1E10C94182EE5E8F5E0712C81918823A9
:1023800021F0739428E17212F9CF66ED71E082EECC
:1023900095E00E94682A4AE050E0672D82EE95E0C1
:1023A0000E94652B80E00E947E0A0E94590B8E01DC
:1023B0000E5F1F4FC12CD12C7601C39466246A9402
:1023C0005C2C0E9470284B015C012091840530E058
:1023D000A0E1B7E20E948E2D9B01AC01C701B601BE
:1023E0000E94B02D20917B0530917C0540917D05A8
:1023F00050917E05620F731F841F951F2091BB05AE
:102400003091BC054091BD055091BE052617370798
:102410004807590718F4F801608229C08C2D0E94E2
:10242000B20961E070E080E090E00E949F28F8012E
:1024300010820E947028681979098A099B09643FF3
:1024400071408105910540F40E94C809F80190810E
:10245000981778F78083EDCF50FE05C05D984198BE
:102460005E9A409A04C05D9A419A5E9840982FEF18
:10247000C21AD20AE20AF20A0F5F1F4F8FEFC81684
:10248000D104E104F10409F09BCFCE019395FC0146
:10249000D82E7FEF68EC2E2F281B271510F051E067
:1024A00056C0DE01129651E02FEF41E03D91321708
:1024B00010F0322F01C0452F5F5F5F3F11F0232FD7
:1024C000F5CF4193242F30E0A1E0B0E0AC0FBD1F69
:1024D000A20FB31F5C93413079F0DE01A20FB31F4E
:1024E0005C93423049F0AFEFBFEFAC0FBD1FA20FBE
:1024F000B31F6C934E3F78F6A2E0B0E0AC0FBD1F67
:10250000A20FB31F7C934D3F30F6A3E0B0E0AC0FB9
:10251000BD1FA20FB31F6C93BECF452F242F30E0F9
:10252000FC01E20FF31F6081AFEFB0E0AC0FBD1F05
:10253000A20FB31F2C91621748F44150DC01A40F85
:10254000B11D2C9120836C934111E8CF5F5F57152B
:1025500020F3372D369520E0231770F4DC01A20F0D
:10256000B11D4C91522F530FFC01E50FF11D50810D
:102570005C9340832E5FF0CFF5E8EF2EF5E0FF2E61
:102580008C01802F8D19871598F4F801C1908F0167
:102590004AE050E06C2D82EE95E00E942E2B6CE21A
:1025A00082EE95E00E943A2AF701C1927F01E9CFBD
:1025B00082EE95E00E94422A81E0CD5EDE4FEFE0A0
:1025C0000C94342E1F920F920FB60F9211241F936A
:1025D0002F933F934F935F936F937F938F939F932B
:1025E000AF93BF93CF93DF93EF93FF93C091860098
:1025F000D091870080918704909188042091A9044C
:10260000211155C09E01281B390B8091BF05909167
:10261000C005A091C105B091C20585FD02C03695E7
:102620002795253C49E03407B8F140910A0150E074
:1026300060E070E02CE1B695A795979587952A956F
:10264000D1F70097A105B10521F481E090E0A0E069
:10265000B0E084179507A607B707D8F480910A0160
:102660008F3FB9F040E080910A01481780F4842F31
:1026700090E0880F991FFC01E757FB4F20813181C3
:10268000FC01E55FFE4F318320834F5FECCF10925A
:10269000AA0410920A010BC02D3B82E0380720F0FB
:1026A00080910A018031D8F08FEF80930A01D09396
:1026B0008804C0938704FF91EF91DF91CF91BF9180
:1026C000AF919F918F917F916F915F914F913F91CA
:1026D0002F911F910F900FBE0F901F901895109182
:1026E0000A0181E0810F80930A01C9010E94DE087E
:1026F000E12FF0E0EE0FFF1FE757FB4F9183808340
:10270000D6CF83E0809380008AE980938100809116
:10271000BF0586FD05C080918100806480938100A3
:102720008FEF9FEF909389008093880080916F00D6
:10273000806280936F0008950E94220D8091D405DD
:10274000843011F41092D40508956F3018F08695F6
:102750008058089589E0689F802D11240895A0E095
:10276000B0E0E5EBF3E10C941F2EC82F0E947C280B
:10277000009138041091390420913A0430913B04BF
:102780006B017C01C01AD10AE20AF30A97018601A3
:1027900049E8C41643E1D406E104F10410F01092B4
:1027A0003C04609338047093390480933A04909306
:1027B0003B042091A9048FEF820F8230D8F5E0917D
:1027C0003C04EE2309F44EC1E13011F482E0B8C1BB
:1027D000E03108F034C181E08E0F80933C04F0E0DA
:1027E000E757FB4FC083803109F0ACC1EBE8F4E060
:1027F000213029F4A181A695A695808108C0808109
:102800009181A92FA695A695A69596958795A03115
:1028100048F4B0E090E0AA0FBB1FA55FBE4F119631
:102820009C938E931092AA04329684E0E939F807BB
:10283000F9F688C1233009F005C1E0913C04E111AB
:1028400004C0CF3009F07EC10DC1E83148F481E009
:102850008E0F80933C04F0E0E857FB4FC08372C1B9
:10286000E83109F0ECC0C111EAC040E050E0ABE053
:10287000CA01B3E0880F991FBA95E1F7A49F9001B0
:10288000A59F300D1124F901E757FB4F6081E181CD
:102890007E2F777075956795FC01EE0FFF1FE55F42
:1028A000FE4F71836083F901E657FB4FB081B69507
:1028B000B695B695E181FE2FF295FF0FF07E6F2F52
:1028C0006B2BE695E695E6957E2F77707595679567
:1028D000FC01EE0FFF1FE35FFE4F71836083F90180
:1028E000E557FB4FB081B295B695B695B370C181EF
:1028F000DC2FDD0FDD0F6D2F6B2BC295C695C695B6
:10290000C370E281E170EE0FEE0F7E2F7C2B759588
:102910006795FC01EE0FFF1FE15FFE4F718360833F
:10292000F901E357FB4FB081B695E181FE2FF79592
:10293000FF27F7956F2F6B2BE6957E2F7770759598
:102940006795FC01EE0FFF1FEF5EFE4F7183608302
:10295000F901E257FB4FB081B295BF70E181FE2FC4
:10296000F295F07F6F2F6B2BE295EF707E2F7770D3
:1029700075956795FC01EE0FFF1FED5EFE4F7183AD
:102980006083F901E157FB4FB081BB1FBB27BB1F21
:10299000C181DC2FDD0F6D2F6B2BCC1FCC27CC1F03
:1029A000E281E370EE0F7E2F7C2B75956795FC011D
:1029B000EE0FFF1FEB5EFE4F71836083F901EF5650
:1029C000FB4FB081B695B695E181FE2FF295FF0FD2
:1029D000FF0FF07C6F2F6B2BE695E6957E2F7770BF
:1029E00075956795FC01EE0FFF1FE95EFE4F718341
:1029F0006083F901EE56FB4F2081229526952770C2
:102A00003181E32FEE0FEE0FEE0F6E2F622B732F3F
:102A100072957695777075956795FC01EE0FFF1F9F
:102A2000E75EFE4F718360834F5F5F4F4230510519
:102A300009F01ECF80919F0483FF1092AA04109288
:102A40003C0480C0243009F07DC060913C046111D9
:102A50000BC0C83AB1F4109275051092740588EA5B
:102A60000E94610681E06CC0613019F4C0933704A4
:102A700004C0623031F4C09336048C2F0E9461068A
:102A80005AC0E09136042E2F30E0220F331F462F1C
:102A900050E0C9010296841795073CF0633268F74D
:102AA000FA01EA57FB4FC083E8CF2D5F3F4F8C2FD1
:102AB00090E060917405709175054217530749F4D1
:102AC000982F8827862797279093750580937405FC
:102AD00032C06817790769F580913704813049F56C
:102AE000E13118F080E180933604F0903604CAE8B2
:102AF000D4E000E010E00F15D0F4FE0131978081A2
:102B000090E0982F88272881822B63E096958795FF
:102B10006A95E1F70E94DE08F801EE0FFF1FE55FFE
:102B2000FE4F918380830F5F1F4F2296E4CF109258
:102B3000AA0410923C0480913C04882319F08F5F12
:102B400080933C04CDB7DEB7E8E00C943B2EE82F31
:102B5000F0E0E654FA4FE185E03150F4F894F0E00B
:102B6000EE0FFF1FE55FFE4F8081918178940895FD
:102B7000E03121F0E13131F483E101C082E10E94D2
:102B8000BE29089580E092E00895A2E2B0E0EBEC67
:102B9000F5E10C94152E9E012F5F3F4F80E1D90186
:102BA0001D928A95E9F764E072E082EE95E029A330
:102BB0003AA30E94682A0E947C0B1D8A1E8A1F8AE3
:102BC000188E312C212C00E0812C912C540170ECBA
:102BD000472E7DE9572E78E5672E75E3772EE0E5E1
:102BE000CE2EE3ECDE2EE12CF12C84EF91E0A0E080
:102BF000B0E08D8F9E8FAF8FB8A380EC97EFAAEBDC
:102C0000B7E3898F9A8FAB8FBC8F80EC9DE9A8E5E5
:102C1000B5E3898B9A8BAB8BBC8B82EE95E00E94DF
:102C20007C2B892B09F4E1C082EE95E00E94A92B50
:102C30009C0133272C32310509F442C0ACF4233215
:102C4000310509F0ABC019821A821B821C821D82D9
:102C50001E821F82188619861A861B861C861D8670
:102C60001E861F86188A60C02434310529F023355A
:102C7000310509F4B2C092C064E482EE95E00E948E
:102C80003A2A2AE030E040EC5DE968E575E382EE3F
:102C900095E00E94C82A6CE282EE95E00E943A2AF2
:102CA0002AE030E040EC57EF6AEB77E382EE95E004
:102CB0000E94C82A6CE282EE95E00E947A2AADCF8B
:102CC0000F5F043009F0A9CF29813A814B815C81E3
:102CD000A8EEB3E00E949D2D698B7A8B8B8B9C8B29
:102CE0002D813E814F8158850E949D2D698F7A8F5D
:102CF0008B8F9C8F29853A854B855C852D8F3E8FE8
:102D00004F8F58A32D853E854F8558890E949D2D54
:102D10006B017C0160323EE473078105910530F45C
:102D200062E38CE10E949F0900E077CF603345E7C2
:102D300074078105910510F462E2F3CF60345CE919
:102D400075078105910510F466E2EBCF80E5C816A2
:102D500083ECD806E104F10410F462E1E2CF90E6DE
:102D6000C9169AEED906E104F10410F465E1D9CF51
:102D7000A0E7CA16A1E1DA06A1E0EA06F10410F420
:102D800061E0CFCFB0EACB16B6E8DB06B1E0EB06E8
:102D9000F10410F463E0C5CF65E0C3CF10ED180F68
:102DA0001A3008F03ACFE1E0F0E0EC0FFD1F24E02C
:102DB000029FE00DF11D1124208131814281538158
:102DC000AAE0B0E00E949D2D610F711D811D911D33
:102DD000608371838283938320CF49885A886B886C
:102DE0007C88812C912C540118CF81149104A1046A
:102DF000B10489F4C301B2010E940E0A61E070E0DF
:102E000080E090E00E949F281D8A1E8A1F8A188EEB
:102E1000312C22242A948D8D9E8DAF8DB8A18816D9
:102E20009906AA06BB06D0F40E94C8092D893E89DE
:102E30004F89588D280F311D411D511D2D8B3E8B03
:102E40004F8B588F381608F4382E821508F4282E28
:102E50003FEF831A930AA30AB30A56C0C301B20113
:102E600028EE33E040E050E00E94D42DBA01A901E1
:102E70002AE030E082EE95E00E941F2B6CE282EEA9
:102E800095E00E943A2A4AE050E0632D82EE95E0F8
:102E90000E942E2B6CE282EE95E00E943A2A6D8908
:102EA0007E898F89988DA50194010E94D42DBA0145
:102EB000A9012AE030E082EE95E00E941F2B6CE22F
:102EC00082EE95E00E943A2A4AE050E0622D82EEBE
:102ED00095E00E942E2B6CE282EE95E00E947A2A09
:102EE0004C0C5D1C6E1C7F1C898D9A8DAB8DBC8D2E
:102EF00084159505A605B70520F449885A886B887E
:102F00007C88812C912C540129893A894B895C89D0
:102F1000283E33404105510509F07FCEA296E2E1FB
:102F20000C94312EACE1B0E0E8E9F7E10C941F2EEF
:102F30000E947C286B017C0181E00E947E0A14E7DC
:102F400003E0198361E0CE0101960E94DB0B009340
:102F500073050E94590B6AEF70E080E090E00E94D8
:102F60009F2880917305833089F482EE95E00E945A
:102F70007C2B892B59F40E947C286C197D098E09C1
:102F80009F096038734C894C9140D8F28091730549
:102F9000833009F44FC08FE70E9477090E948A09A5
:102FA0008983843511F083E05CC00E948A09109205
:102FB0004605809347050E948A0920914605309175
:102FC0004705280F311D30934705209346050E9481
:102FD0008A09809348050E948A09809349058131B6
:102FE00010F7F12C0F2D10E08091490590E0880F2B
:102FF000991F0817190740F40E948A09F801E65B37
:10300000FA4F8083F394EECF80E7898361E0CE01AD
:1030100001960E94DB0B83E0809373050E94590B9D
:1030200062E370E080E090E00E949F288091730549
:10303000833011F482E015C08FE70E9477090E9467
:103040008A098983803509F0AECF0FE915E00E9427
:103050008A09F80181938F01F5E00A3B1F07B9F750
:1030600081E06C96E8E00C943B2E80914505992711
:1030700087FD9095A92FB92FFC013196EB30F10512
:1030800008F066C0EC5CFF4F0C944C2E62E778E0D1
:1030900082EE95E00E94562A80E893E00E94300C70
:1030A0006AE578E082EE95E00E94562A65E378E0D2
:1030B00082EE95E00E94562A6BE078E082EE95E081
:1030C0000E94562A6AEE77E082EE95E00E94562A28
:1030D0006DEB77E082EE95E00E94562A67E977E093
:1030E00082EE95E00E94562A63E777E082EE95E053
:1030F0000E94562A6CE477E082EE95E00E94562A00
:1031000082EE95E00E94422A0E94630D21C06FE288
:1031100077E01AC06AE077E017C065EF76E014C088
:1031200066ED76E011C062E976E00EC06DE776E00C
:103130000BC068E676E082EE95E00E94562A62E2D5
:1031400076E002C06CE076E082EE95E00E94562ABE
:103150006AE070E080E090E00E949F2882EE95E0B7
:103160000E947C2B892B29F082EE95E00E94A92BEE
:10317000F5CF0895ACE1B0E0E0ECF8E10C941F2E3F
:10318000909145059F3F09F023C1482F50E0FA0177
:103190003A97EF36F10508F00FC1E15CFF4F0C9450
:1031A0004C2E61E172E0A0C06DE172E082EE95E02C
:1031B0000E94682A85E789838BE1EFE9F5E0DE016B
:1031C000129601900D928A95E1F76CE1CE0101967D
:1031D0000E94DB0B0E94590B83E08093730568EC1F
:1031E00070E080E090E00E949F2880917305843019
:1031F00009F0E2C08FE70E9477090E948A0989835B
:10320000853509F0D9C06DEE74E082EE95E00E943C
:10321000562A6FEC74E082EE95E00E94562A61EB2C
:1032200074E096C065E372E082EE95E00E94682A41
:1032300089E6898361E0CE0101960E94DB0B0E9442
:10324000590B83E08093730568EC70E080E090E0B8
:103250000E949F2880917305843009F0ADC08FE7EC
:103260000E9477090E948A0989838E010E5F1F4F91
:103270007E014DE1E40EF11C0E948A09F801819360
:103280008F01EE15FF05C1F78BE1FE013296AFE924
:10329000B5E001900D928A95E1F78981893409F0B2
:1032A0008BC063E974E082EE95E00E94562A65E7E0
:1032B00074E082EE95E00E94562A67E574E048C00B
:1032C0006FE472E082EE95E00E94682A8EEF8093B0
:1032D000450572C0805287508053909148059817D9
:1032E00008F066C06EE572E082EE95E00E94682A02
:1032F00063C084E18093450560E274E029C085E104
:103300008093450569EE73E023C086E1809345050F
:1033100062EB73E01DC087E18093450568E673E0CA
:1033200017C088E18093450567E573E011C089E126
:103330008093450563E473E00BC08AE18093450503
:103340006EE273E005C08BE18093450566E073E0B3
:1033500082EE95E00E94562A2FC06CEE72E082EE5B
:1033600095E00E94562A8091AD0591E01DC066ED62
:1033700072E082EE95E00E94562A8091AD0592E0BF
:1033800013C061EC72E082EE95E00E94562A8091B3
:10339000AD0594E009C066EA72E082EE95E00E9415
:1033A000562A8091AD0598E089278093AD058FEF6F
:1033B000809345050E94041082EE95E00E947C2BCC
:1033C000892B09F45BC182EE95E00E94A92BF4CF12
:1033D0000E940311882309F451C18091DF048111F7
:1033E00004C08FEF8093450541C140E050E060E0AC
:1033F00070E080EE94E00E94C32E40914505042FBA
:10340000112707FD1095212F312FF8013197EB314E
:10341000F10508F01BC1E255FF4F0C944C2E5527C7
:1034200047FD50952091480530E0241735070CF4EE
:103430000DC18B019C010150110921093109003294
:1034400011052105310558F0C0904905EBE4F5E080
:10345000F12CD12CA8E2EA2E415051090FC0FA01FB
:10346000E156FA4F61506083D9C0DF0111972C916A
:1034700030E02417350729F0F3943296FC10F5CF8D
:10348000CBC00E2D10E020E030E00617170728070C
:10349000390741F42081DA01A156BA4F11962C93D5
:1034A000DD24D394E394E8CF6F3F71058105910546
:1034B00011F008F0CBC06093B705B0C06F3F710545
:1034C0008105910511F008F0C1C06093B805A6C050
:1034D0006F3F71058105910511F008F0B7C0609349
:1034E000B9059CC02091E00420622037E9F440E057
:1034F00050E060E070E081EE94E00E94C32E9B01FA
:10350000AC01DC01CB010197A109B1090897A10524
:10351000B10508F0AEC0A4EDB0E30E949D2D6A5E37
:103520007C4A8A46954E24C02636E9F440E050E0B5
:1035300060E070E081EE94E00E94C32E9B01AC013C
:10354000DC01CB010197A109B1090797A105B105DC
:1035500008F08FC0A8EAB1E60E949D2D645E7C430E
:103560008E46944E05C0611571058105910579F06F
:103570008B019C01005C1D49284535430130FAE56B
:103580001F07F2E62F07F2E03F0708F05FC06093E5
:10359000AF057093B0058093B1059093B2053EC01E
:1035A0006F3F71058105910511F008F04FC06093E0
:1035B000B30534C08B019C01015011092109310967
:1035C0000F3F11052105310508F040C06093B40597
:1035D00025C08B019C01045C1940210931090D347F
:1035E0004DE114072105310528F47093B605609369
:1035F000B50514C0611571058105910521F48FEFA2
:103600008093AE050BC06134710581059105F0F41E
:1036100061506093AE0502C0DD20C1F08091DE04F0
:1036200081111AC080917F0590918005A09181053C
:10363000B09182050196A11DB11D80937F059093E5
:103640008005A0938105B093820506C060E772E013
:1036500082EE95E00E94682A0E94F9108FEF809315
:1036600045056AE082EE95E00E947A2A0E940410E5
:1036700005C061E070E080E090E07ACF6C96E8E011
:103680000C943B2E6AE572E082EE95E00E94562A89
:1036900062E472E082EE95E00E94562A82EE95E0A6
:1036A0000E947C2B892B31F082EE95E00E94A92BA1
:1036B0000E94BA180E949217823029F0833051F488
:1036C0006DE072E002C064E272E082EE95E00E947A
:1036D000562A08958FEF809345051092DE040E94CC
:1036E0000410809145058E3F69F082EE95E00E94BE
:1036F0007C2B892BB1F382EE95E00E94A92B0E94CE
:10370000BA18EFCF08950F931F93109145051F3FEF
:1037100009F0D2C0893409F457C000F5883309F4A0
:1037200069C058F4803309F477C008F061C08B3168
:1037300009F440C08132B1F1B9C0813409F487C0C5
:1037400030F4893309F466C0803461F1AFC082344B
:1037500009F48EC0863409F448C0A8C0823609F442
:1037600087C078F4883531F128F48235C1F183358A
:10377000E1F09CC08A3509F494C0813609F467C031
:1037800095C0823761F128F4863679F18936E1F007
:103790008DC0883779F08A3709F483C0833709F000
:1037A00085C003C061E172E015C00E94340D6EE86F
:1037B00072E004C00E943D0D68EA72E082EE95E07E
:1037C0000E94682A8EEF70C00E947A060E94BF068F
:1037D00067EC72E082EE95E00E94682A67C081E0A3
:1037E0000E94DF0660EE72E0F5CF0E94AE105EC070
:1037F00080535AC06AEF71E082EE95E00E94562A2B
:1038000090919E0588E0890F8871977E892B80931F
:103810009E051AC089E048C067EE71E082EE95E02F
:103820000E94562A8091BF059091C005A091C105C4
:10383000B091C20520E182278093BF059093C00517
:10384000A093C105B093C205109345052FC061ED4B
:1038500071E082EE95E00E94562A8091BF0590911A
:10386000C005A091C105B091C20540E4842710C0F5
:1038700060EC71E082EE95E00E94562A8091BF05CF
:103880009091C005A091C105B091C20520E28227A8
:103890008093BF059093C005A093C105B093C20566
:1038A00002C00E94421B8FEF809345058091450521
:1038B0008E3F09F0D4C0DDC00E940311882309F4B3
:1038C000D8C08091DF04811104C08FEF809345053B
:1038D000C6C040E050E060E070E080EE94E00E94FE
:1038E000C32E00914505112707FD1095212F312F7B
:1038F000F8013197E930F10508F0B4C0E753FF4F04
:103900000C944C2E8B019C01015C1D4928453543CC
:103910000F3F19452246324008F0A4C060937B0552
:1039200070937C0580937D0590937E0577C06093AE
:103930007F0570938005809381059093820581E0D7
:103940008093DE046BC0683071058105910508F035
:1039500089C06093830562C08B019C0101501109ED
:10396000210931090A3011052105310508F07AC015
:103970006093840553C061EB71E080EE94E00E9497
:10398000FD2F10E0009799F00E94D72F009779F053
:10399000183130F4E12FF0E0EA58FA4F87871F5FC3
:1039A00061EB71E080E090E00E94FD2FEBCF1831D9
:1039B000A8F5E12FF0E0EA58FA4F17861F5FF7CF1E
:1039C000653071058105910508F04CC060939D0537
:1039D00025C08B019C0101501109210931090630D4
:1039E000110521053105F0F520919E05287F262B34
:1039F00020939E0513C08B019C01015011092109E0
:103A000031090115124C2140310560F560937705AD
:103A1000709378058093790590937A058091DE0400
:103A2000811113C080917F0590918005A09181053F
:103A3000B09182050196A11DB11D80937F059093E1
:103A40008005A0938105B09382050E94F9108FEF45
:103A5000809345056AE082EE95E00E947A2A0E94F2
:103A6000351807C060E772E082EE95E00E94682A90
:103A7000ECCF1F910F9108958FEF80934505109221
:103A8000DE040E943518809145058E3F69F082EE74
:103A900095E00E947C2B892BB1F382EE95E00E9489
:103AA000A92B0E94831BEFCF6AE070E080E090E0DA
:103AB0000E949F2882EE95E00E947C2B892B29F0A2
:103AC00082EE95E00E94A92BF5CF0895CF93C82FE1
:103AD000682F82EE95E00E94D62B90916A059C2774
:103AE00090936A05CF910895A1E0B0E0EAE7FDE187
:103AF0000C94252E99830E94661D9981892F0E941E
:103B0000661D2196E2E00C94412E1F93CF93DF9324
:103B1000182FEB0110926A0565EB70E082EE95E0DC
:103B20000E94590662E670E082EE95E00E94590616
:103B3000812F0E94661DCE010E94741DDF91CF91DE
:103B40001F91089560916A0582EE95E00E94D62B40
:103B50000895A1E2B0E0EFEAFDE10C94212E7B0193
:103B60008A018C3009F453C108F040C0863009F452
:103B7000BCC018F5833009F491C070F4813009F4A9
:103B800072C0823009F048C26BE170E082E00E94AE
:103B9000851D0FE915E078C0843009F487C08530B1
:103BA00009F03AC26091490570E0660F771F85E021
:103BB0000E94851D0AE415E086C0893009F4A7C07B
:103BC00070F4873009F49BC0883009F025C261E0A9
:103BD00070E088E00E94851D8091D40523C28A3060
:103BE00009F4CAC08B3009F4F2C016C28A3609F44F
:103BF00075C1D8F4873609F43AC138F4853609F42A
:103C00000EC1863609F41FC107C2883609F437C1D0
:103C1000893609F001C261E070E089E60E94851DE5
:103C20000E947A060E94BF06F5C18D3609F4D4C100
:103C300038F48B3609F491C18C3609F49AC1ECC181
:103C40008E3609F4DCC1873C09F0E6C161E070E022
:103C500087EC0E94851D81E00E94661D0E94A21DC6
:103C600010926B05E3C169E270E081E00E94851D5E
:103C700006E715E0F80181918F010E94661DF5E0CD
:103C80000F391F07B9F7D0C1F80181918F010E9448
:103C9000661DF5E00A3B1F07B9F7C6C161E070E099
:103CA00083E00E94851D0E949217BCC161E070E014
:103CB00084E00E94851D81E00E94661D0E94A21D75
:103CC0000E94C515B3C18091490590E0880F991FE6
:103CD00098012A5435402817390708F0A5C1F80182
:103CE00081918F010E94661DEECF62E070E086E058
:103CF0000E94851D80E893E00E94741D95C161E0DB
:103D000070E087E00E94851D809148058BC186E6A2
:103D1000898361E0CE0101960E94DB0B0E94590B62
:103D200083E08093730568EC70E080E090E00E948F
:103D30009F28809173058430D9F48FE70E9477091A
:103D40000E948A098983863469F460E270E089E020
:103D50000E94851D10E20E948A090E94661D115072
:103D6000D1F762C161E070E089E00E94851D52C117
:103D700061E070E089E053C169E170E08AE00E948F
:103D8000851D82E08093BA05209172058091BF0560
:103D90009091C005A091C105B091C205222311F0F8
:103DA000806801C08F778093BF059093C005A09372
:103DB000C105B093C2050AEB15E0F80181918F01AE
:103DC0000E94661DF5E0033D1F07B9F72DC161E2B2
:103DD00070E08BE00E94851D8091AA048F3F39F02E
:103DE0008091AA0491E0980F9093AA0402C0809158
:103DF000AA040E94661D10E0812F0E94A7150E9450
:103E000009090E94741D1F5F1031B1F70DC161E0F7
:103E100070E08CE00E94851D8091D30503C161E0B4
:103E200070E085E60E94851D89E2E816F10409F03C
:103E3000F8C0D801E6E7F5E08D91819385E0EF3990
:103E4000F807D1F7E7C061E070E086E60E94851DC3
:103E5000EBE1EE16F10409F0E4C0D801EFE9F5E07A
:103E60008D91819385E0EA3BF807D1F7D3C061E0FB
:103E700070E087E60E94851D0E94340DCBC061E092
:103E800070E088E60E94851D85E789838BE1EFE974
:103E9000F5E0DE01129601900D928A95E1F76CE152
:103EA000CE0101960E94DB0B0E94590B83E08093A8
:103EB000730560E273E080E090E00E949F288091AB
:103EC0007305843009F0ADC08FE70E9477090E9426
:103ED0008A098983853509F0A4C09CC061E070E03F
:103EE0008AE60E94851D89E6898361E0CE010196FC
:103EF0000E94DB0B0E94590B83E08093730560E204
:103F000073E080E090E00E949F28809173058430E8
:103F100009F087C08FE70E9477090E948A09898388
:103F20008E010E5F1F4F7E01EDE1EE0EF11C0E942F
:103F30008A09F80181938F01EE15FF05C1F78BE126
:103F4000FE013296AFE9B5E001900D928A95E1F756
:103F50008981893409F065C05DC061E070E08BE65D
:103F60000E94851DF80180818093D4050E943D0D3B
:103F700051C061E070E08CE60E94851DF0E2EF1612
:103F8000F10461F487E6898380E2F801DE0112968C
:103F900001900D928A95E1F761E203C087E489837D
:103FA00061E0CE0101960E94DB0B0E94590B83E079
:103FB000809373056CE474E080E090E00E949F2899
:103FC00080917305843069F58FE70E9477090E941C
:103FD0008A09873431F51EC061E070E08DE60E94E9
:103FE000851D89E1E816F104E1F4D801EAEBF5E07A
:103FF0008D91819385E0E33DF807D1F70BC061E037
:1040000070E08EE60E94851DF80180818093D305C3
:104010000E941D0D81E006C061E070E08AEC0E9404
:10402000851D80E00E94661D0E94A21DA196E6E00B
:104030000C943D2EA0E0B0E0E0E2F0E20C941F2EE4
:10404000CAECD3E014E606E035E0F32E44E0E42EBB
:1040500053E0D52E62E0C62E82EE95E00E947C2BC6
:10406000892B09F49BC082EE95E00E94A92B282F92
:10407000809335044091340450E04730510560F797
:10408000FA01EE52FF4F0C944C2E853B29F781E04C
:1040900080933404E1CF823609F07DC0C0923404AD
:1040A000DBCF8093330480933204D0923404D4CF96
:1040B0009C013327309331042093300490913204D3
:1040C000982790933204E0923404C6CF382F2227E9
:1040D0004091300450913104242B352B309331041E
:1040E0002093300490913204982790933204F092F8
:1040F00034042536310508F4AFCF61E070E08CEC74
:104100000E94851D81E00E94661D0E94A21D43C081
:1041100020912E0430912F04F901E653FC4F808347
:1041200090913204982790933204C901019690939C
:104130002F0480932E042091300430913104821793
:10414000930708F489CF0093340486CF809132041A
:1041500082130BC060912E0470912F044AEC53E03F
:10416000809133040E94A91D0DC062E070E08BECC9
:104170000E94851D809133040E94661D80916A050E
:104180000E94661DFE01812F11928A95E9F7109217
:104190002F0410922E04109234045ECFCDB7DEB7F8
:1041A000E8E00C943B2E81E080936B0580916B05D9
:1041B000882349F082EE95E00E947C2B892BB1F395
:1041C0000E941A20F3CF0895AAE2B0E0EAEEF0E2EE
:1041D0000C941D2E0E9470286B017C0181E00E94CE
:1041E0007E0A82EE95E00E947C2B892B29F082EEDC
:1041F00095E00E94A92BF5CF5E98409811E072E6F9
:10420000B72EE9E2AE2E03E00E9470286C197D09FA
:104210008E099F09693C710581059105E0F1112323
:10422000D1F10E9470286B017C015D9A419A80ED6A
:1042300097E00E94A807B982E6E7F5E0DE01129652
:104240008A2D01900D928A95E1F76AE2CE010196DE
:104250000E94DB0B5D98419880E090E00E94A807E7
:10426000009373050E94590B62E370E080E090E0D8
:104270000E949F2880917305843061F40093730538
:104280008FE70E9477090E948A0911E0823419F4AD
:1042900010E001C011E083E10E949529892BA1F46F
:1042A00011E012C05E9A409A5D9A419A82EE95E0C2
:1042B0000E94A92B8D309105B9F06CF40A97A1F0FA
:1042C0005E9840985D98419882EE95E00E947C2B24
:1042D000892B41F799CF8332910579F0823491058A
:1042E00079F70E94D320ECCF62EB71E082EE95E08B
:1042F0000E94562A0E943C1DE3CF0E94C515E0CFC4
:104300008F929F92AF92BF92CF92DF92EF92FF92E5
:104310001F93CF93DF9383E10E949529892B09F0A6
:1043200089C068EC70E080E090E00E949F2880E007
:1043300090E00E94A8070E9470284B015C016B016D
:104340007C0180ECC80E82E1D81EE11CF11C0E94A9
:1043500070286C157D058E059F0530F483E10E9461
:104360009529892BA1F364C083E10E949529892BAB
:1043700009F05EC080ED97E00E94A8070E947028B7
:104380006B017C01D0E0C1E088E4880E86E2981ED3
:10439000A11CB11C11E083E10E949529892B21F514
:1043A0008C149D04AE04BF0430F480ED97E00E94AD
:1043B000A807D1E0F0CF0E9470286C197D098E0902
:1043C0009F09693C71058105910528F30E947028B9
:1043D0006B017C01C12719F080ED97E002C080E0FD
:1043E00090E00E94A807D7CF80E090E00E94A80745
:1043F000DD23B9F08091D30590E0019665E070E08F
:104400000E94C02D8093D3050E941D0D0E949C1315
:104410000E943D0D64EF71E080E090E00E949F28D3
:1044200009C080E00E94DF060E94B5110E94340D91
:104430000E94E420DF91CF911F91FF90EF90DF90D9
:10444000CF90BF90AF909F908F900895CF92DF92C2
:10445000EF92FF9280E00E94DA070E94B10761E0CC
:1044600086E00E94292961E085E00E94292961E017
:104470008EE00E94292961E08FE00E94292960E0F6
:1044800083E10E94292960E088E00E94292961E0F7
:1044900088E00E9462290E949F0740E052EC61E0A0
:1044A00070E082EE95E00E94C42C0E949C130E9452
:1044B0003D0D0E9481138FEF8093AA040E94C607CE
:1044C00078940E9470286B017C018091AA048F3F30
:1044D00059F40E9470286C197D098E099F09603D6E
:1044E00077408105910588F380ED97E00E94A80749
:1044F00061E083E10E9462295E9A409A82EE95E033
:104500000E947C2B892B29F082EE95E00E94A92B3A
:10451000F5CF6DEF72E082EE95E00E94372A80E8D9
:1045200093E00E94300C64E173E082EE95E00E941B
:10453000372A4AE050E069E070E082EE95E00E94A0
:10454000072B62E370E080E090E00E949F2882EEFB
:1045500095E00E947C2B04970CF182EE95E00E947E
:10456000A92B82349105D1F482EE95E00E94A92B0B
:104570008E34910599F482EE95E00E94A92B843443
:10458000910561F482EE95E00E94A92B819731F4A8
:1045900080E090E00E94A8070E94E4204091770507
:1045A000509178056091790570917A05DB01CA0117
:1045B0000197A109B1090497A105B10568F44093D9
:1045C000A904433029F440EA56E861E070E004C0F1
:1045D00040E052EC61E070E082EE95E00E94C42C75
:1045E0000E9480215E98409880E090E00E94A80799
:1045F0000E9481131092C5048091BF0583FF11C0F2
:1046000080918B05882351F080919205882331F0A9
:1046100080919905882311F087E001C085E080939F
:10462000C50480E00E947E0A8091C6040E94B209FF
:104630000E94590B10923F0410923E0410923D04C8
:10464000F12C8091D4058F15B0F062E370E080E02A
:1046500090E00E949F2880ED97E00E94A80762E307
:1046600070E080E090E00E949F2880E090E00E944F
:10467000A807F394E6CF80919E0584FF08C0982F89
:10468000987181E0983109F080E00E9471118FE00B
:104690000E94DA07FF90EF90DF90CF900895EF929D
:1046A000FF920F931F93CF93DF938C016EE770E01F
:1046B00082EE95E00E945906E801F12CF0E2EF2E1F
:1046C0008E0188818D57823048F46DE770E082EE6C
:1046D00095E00E94590688818E2588832196F801ED
:1046E000608182EE95E00E94D62BF394F9E0FF12F0
:1046F000E7CF6EE770E082EE95E00E945906CDB7F5
:10470000DEB7E6E00C943D2EA9E0B0E0EAE8F3E283
:104710000C94252E9091C70491110EC09EEF9983A1
:104720008A836B8350E0559547954C832D8319867A
:1047300018861F821E822EC04091CC04842F90E0E8
:10474000B4E095958795BA95E1F7242F2F7030E066
:104750008217930719F18DEF89831B82FE0134962E
:1047600050E0842F90E0A4E095958795AA95E1F715
:10477000242F2F7030E08217930749F0DC01A353F8
:10478000BB4F8C918193405F5F5F563051F74093F0
:10479000CC045A83CE0101960E944F238091C70416
:1047A00090E0019666E070E00E94C02D8093C704FF
:1047B0002996E2E00C94412EA0E0B0E0E2EEF3E2B4
:1047C0000C941E2E6C016EE770E082EE95E00E9464
:1047D00059068601E12CF12CC0E0D0E030E2B32E86
:1047E000F801608183E8860F823078F46DE770E02D
:1047F00082EE95E00E945906F80160816B2570E019
:1048000082EE95E00E94590604C082EE95E00E9477
:10481000D62BE114F10459F0F80180819E01280F94
:10482000311DC901C92FDD27C80FD91FDD273FEF73
:10483000E31AF30A89E0E816F10459F028E0E216D9
:10484000F10421F48C2F8095F60180870F5F1F4FB4
:10485000C7CFCDB7DEB7E9E00C943A2EA9E0B0E0BF
:10486000E4E3F4E20C94252EE82F362F8091C70460
:1048700090E0019664E270E00E94C02D8093C7042E
:1048800058E9598350E15A83813089F048F08230E9
:10489000B9F08330D9F48B8381EF8C833D8319C0C9
:1048A00085E08B8381EF8C832F5F2D8312C08B83F8
:1048B00081EF8C8384E6489FA00111245D8309C0A9
:1048C00084E08B8381EF8C83ED8303C00E94AE1163
:1048D00004C0CE0101960E94DC232996E2E00C94EC
:1048E000412EA2E0B0E0E7E7F4E20C941A2E182F74
:1048F000762E2A8349830E947C286B017C0180915B
:10490000DD048090C8049090C904A090CA04B090BF
:10491000CB042A8149818823C1F0D701C6018819B7
:104920009909AA09BB094C015D0191EE89169EE225
:104930009906A104B10420F1241708F4422F202F76
:10494000672D812F0E942E2413C0D701C60188191C
:104950009909AA09BB094C015D0191E3891695E704
:104960009906A104B10460F0672D812F0E94842371
:10497000C092C804D092C904E092CA04F092CB0459
:104980002296EDE00C94362EA2E2B0E0EAECF4E2DE
:104990000C941B2E8CE00E94990981110FC06CE1D0
:1049A00073E082EE95E00E94682A5E9A409A80E069
:1049B0000E947E0A0E94590B5E98409882EE95E014
:1049C0000E947C2B892B01F182EE95E00E94A92B9D
:1049D0009091A904992319F00E94AF13EFCF409151
:1049E0003E0450E09A012F5F3F4F2F7133276091B3
:1049F0003F0470E02617370709F3FA01E75BFB4F26
:104A0000808320933E04DACF80917305843009F0CF
:104A100086C00E947C28611571058105910549F0C9
:104A20006093B7047093B8048093B9049093BA0468
:104A30000CC081E090E0A0E0B0E08093B7049093D8
:104A4000B804A093B904B093BA048091AD049091D6
:104A5000AE0481609093AE048093AD0483E08093B4
:104A600073058FE70E94770909E614E00E948A091E
:104A7000F80181938F01F4E002371F07B9F7209105
:104A8000720480916904982F922796FF3BC090E4AE
:104A9000922790937204982F98739833F1F410E052
:104AA000212F30E080916904877090E0821793078E
:104AB0004CF11F5F20919E05812F90E0FC01E7598A
:104AC000FB4F24FF04C080810E949011E9CF6081D8
:104AD00082EE95E00E94D62BE3CF8F7399F48091FC
:104AE0006A048093B60480916B048093B40480912F
:104AF0006C048093B30480916F0490E09093AC04B5
:104B00008093AB0480913D04813019F482E080935E
:104B10003D0480913D04833011F410923D040E94C5
:104B20007C286B017C018091AF049091B004A0912E
:104B3000B104B091B2040097A105B105C9F0A70175
:104B40009601281B390B4A0B5B0BDA01C901883B24
:104B50009B40A105B10560F00E94C8098093B5048F
:104B60001092AF041092B0041092B1041092B204EB
:104B70008091BB049091BC04A091BD04B091BE048F
:104B800046015701881A990AAA0ABB0A86E795E0E6
:104B90000E94F40786169706A806B90608F4A9C06D
:104BA000C092BB04D092BC04E092BD04F092BE045B
:104BB0000E9457068091AA048830A0F08091BF051A
:104BC0009091C005A091C105B091C2056CE1B69568
:104BD000A795979587956A95D1F7892B8A2B8B2B6B
:104BE00009F0A8C18091AA048F5F8093AA048091E4
:104BF000B7049091B804A091B904B091BA04009799
:104C0000A105B105F1F0C81AD90AEA0AFB0A86E73C
:104C100095E00E94F4076C157D058E059F0508F050
:104C200008C18091BF0584FD04C080ED97E00E941B
:104C3000A8071092B7041092B8041092B904109209
:104C4000BA0490917204907C9093720450913E0447
:104C500080913F0420913D04581709F407C1223088
:104C600009F004C1905890937204E0919E05E7709A
:104C7000F0E0E658FC4F6081693008F0DFC0615019
:104C800040E04613DDC080933F0487E3840F90919A
:104C90007204892B809372044093400483E08093D4
:104CA0003D045D9A419A809183059091C5049111CC
:104CB00032C10E94790A8091C6040E94B209E09133
:104CC0009E05E770F0E0E658FC4F608182E794E0D3
:104CD0000E94940BE091C604EF5FE093C604E831B4
:104CE00009F425C1F0E0EA58FA4F8785882309F4D2
:104CF0001EC10E94030C813069F580919E05887168
:104D000049F18091AD049091AE04880F991F909362
:104D1000AE048093AD0483E0809373050E94590B29
:104D20000E947C286093AF047093B0048093B10418
:104D30009093B204672B682B692B61F481E090E0BB
:104D4000A0E0B0E08093AF049093B004A093B104CE
:104D5000B093B20480919E0584FF1FC08091AD0482
:104D60009091AE048E7F0E942A09182F6091AB04A7
:104D70008091B6040E94A513482F612F8091B5043D
:104D800049A30E94A5130091D405282F49A1609141
:104D9000B3048091B4040E9471245D98419880917D
:104DA000C3048130C1F018F08230B1F1D1C083E189
:104DB0000E949529892B09F0CBC081E08093C30420
:104DC0000E9470286093BF047093C0048093C10454
:104DD0009093C204BDC083E10E949529892B31F5CF
:104DE0000E947028C090BF04D090C004E090C1041D
:104DF000F090C2046C197D098E099F09693E7340C9
:104E00008105910508F4A4C082E08093C30480ED7D
:104E100097E00E94A8079CC083E10E949529892BF6
:104E200009F496C080E090E00E94A8071092C304A5
:104E30008FC080E090E00E94A80703CF68E020CFF9
:104E4000851709F420CF4F5F242F30E090E0F9015F
:104E5000EE58FB4FDC01A75BBB4F7C917083F901DF
:104E6000E05CFB4F708301968F710BCF2430B1F45F
:104E70002091400481E494E0A3E7B4E0FC013E2FDC
:104E8000381B321718F431913D93F9CF87E3820F25
:104E900090917204892B8093720400CF8091C30497
:104EA000823071F49160909372045E9A409A53EC50
:104EB000E52E55E0F52E8E010F5F1F4FB80111C092
:104EC0005E98409880913D04811103C081E08093F9
:104ED0003D0480913D04833051F784E080933D048C
:104EE000E6CFF70181917F0169A37AA30E94A715FC
:104EF000F801819391938F0169A17AA1F3EDEF16E7
:104F0000F5E0FF0671F780919E0543E754E0877056
:104F10000E947908C6CE882309F4CBCE2091C40420
:104F200031E0320F3093C4042913C3CE0DC0109268
:104F3000C604DFCE8091AA04883011F45E9A409AAC
:104F400089E08093AA04D5CE1092C4048150B1CEDA
:104F5000A296ECE00C94372E8230E8F4E82FF0E0D3
:104F6000EE0FFF1FEB52FA4F71836083813041F0E7
:104F7000809169008C7F842B80936900E89A089562
:104F800080916900440F551F440F551F837F842B68
:104F900080936900E99A08951F920F920FB60F92BD
:104FA00011242F933F934F935F936F937F938F932E
:104FB0009F93AF93BF93EF93FF938091D50590910B
:104FC000D605892B29F0E091D505F091D6050995F4
:104FD000FF91EF91BF91AF919F918F917F916F91D1
:104FE0005F914F913F912F910F900FBE0F901F90A7
:104FF00018951F920F920FB60F9211242F933F9383
:105000004F935F936F937F938F939F93AF93BF93D0
:10501000EF93FF938091D7059091D805892B29F0C4
:10502000E091D705F091D8050995FF91EF91BF91D7
:10503000AF919F918F917F916F915F914F913F9130
:105040002F910F900FBE0F901F9018951F920F92E7
:105050000FB60F9211242F933F938F939F93AF938B
:10506000BF938091DA059091DB05A091DC05B091AA
:10507000DD053091D90523E0230F2D3720F401966B
:10508000A11DB11D05C026E8230F0296A11DB11D6B
:105090002093D9058093DA059093DB05A093DC0576
:1050A000B093DD058091DE059091DF05A091E005CC
:1050B000B091E1050196A11DB11D8093DE0590938D
:1050C000DF05A093E005B093E105BF91AF919F91FB
:1050D0008F913F912F910F900FBE0F901F901895B9
:1050E0002FB7F8946091DA057091DB058091DC05AB
:1050F0009091DD052FBF08953FB7F8948091DE05AC
:105100009091DF05A091E005B091E10526B5A89B3F
:1051100005C02F3F19F00196A11DB11D3FBF6627A5
:10512000782F892F9A2F620F711D811D911D42E0EA
:10513000660F771F881F991F4A95D1F70895CF9260
:10514000DF92EF92FF92CF93DF936B017C010E947D
:105150007C28EB01C114D104E104F10479F00E9430
:105160007C286C1B7D0B683E7340A0F381E0C81A5D
:10517000D108E108F108C851DC4FECCFDF91CF91A5
:10518000FF90EF90DF90CF900895789484B582607F
:1051900084BD84B5816084BD85B5826085BD85B5DB
:1051A000816085BDEEE6F0E0808181608083E1E88A
:1051B000F0E01082808182608083808181608083C2
:1051C000E0E8F0E0808181608083E1EBF0E08081C5
:1051D00084608083E0EBF0E0808181608083EAE797
:1051E000F0E0808184608083808182608083808120
:1051F000816080838081806880831092C1000895DF
:10520000833081F028F4813099F08230A1F0089544
:105210008630A9F08730B9F08430D1F480918000D5
:105220008F7D03C0809180008F77809380000895E8
:1052300084B58F7702C084B58F7D84BD0895809139
:10524000B0008F7703C08091B0008F7D8093B00055
:105250000895CF93DF9390E0FC01ED50F44F24913B
:10526000FC01E95FF34F8491882349F190E0880FB6
:10527000991FFC01E15DF34FA591B4918B5D934FB4
:10528000FC01C591D4919FB7611108C0F8948C912D
:10529000209582238C93888182230AC0623051F446
:1052A000F8948C91322F309583238C938881822BB4
:1052B000888304C0F8948C91822B8C939FBFDF91DC
:1052C000CF910895A1E0B0E0E8E6F9E20C94232E36
:1052D000282F30E0F901E152F44F8491F901ED50AB
:1052E000F44F1491F901E95FF34F04910023C9F0E1
:1052F000882321F069830E9400296981E02FF0E072
:10530000EE0FFF1FEB5DF34FA591B4919FB7F8949B
:105310008C91611103C01095812301C0812B8C9366
:105320009FBF2196E4E00C943F2ECF93DF93282F6C
:1053300030E0F901E152F44F8491F901ED50F44F5E
:10534000D491F901E95FF34FC491CC2391F081111D
:105350000E940029EC2FF0E0EE0FFF1FE55EF34FF7
:10536000A591B4912C912D2381E090E021F480E06F
:1053700002C080E090E0DF91CF9108958E3008F078
:105380008E50877020919D0190E4299F90011124F7
:10539000822B80937C0080917A00806480937A00D5
:1053A00080917A0086FDFCCF809178002091790071
:1053B00090E0922B0895A0E0B0E0E1EEF9E20C94C9
:1053C0001F2E6C017A01EB01E60EF71E00E010E0E3
:1053D000CE15DF0561F06991D601ED91FC91019048
:1053E000F081E02DC6010995080F191FF1CFC80102
:1053F000CDB7DEB7E8E00C943B2E6115710589F05E
:10540000DB010D900020E9F7AD0141505109461B29
:10541000570BDC01ED91FC910280F381E02D0995A1
:10542000089580E090E00895EF92FF920F931F930C
:10543000CF93DF938C01FB01C0E0D0E064917F014A
:105440008FEFE81AF80A662361F0D801ED91FC911C
:105450000190F081E02DC8010995C80FD91FF7010F
:10546000EDCFCE01CDB7DEB7E6E00C943D2E0E9425
:10547000FD290895DC01ED91FC910190F081E02D72
:10548000099508950F931F93CF93DF93EC016DE07F
:105490000E943A2A8C016AE0CE010E943A2A800FCB
:1054A000911FDF91CF911F910F9108950F931F933B
:1054B000CF93DF93EC010E94142A8C01CE010E944D
:1054C000422A800F911FDF91CF911F910F91089574
:1054D0000F931F93CF93DF93EC010E94FD298C0162
:1054E000CE010E94422A800F911FDF91CF911F9120
:1054F0000F9108950F931F93CF93DF93EC010E94B8
:105500003A2A8C01CE010E94422A800F911FDF911E
:10551000CF911F910F910895A1E2B0E0E2E9FAE284
:105520000C941B2E7C01C42EE52FCB01D22E19A288
:1055300021E02D1510F02AE0D22E8E010F5D1F4FB5
:105540008D2C912CA12CB12C6C2D7E2FA5019401BA
:105550000E94D42D8C2DD29E801911240150110946
:105560008A3010F4805D01C0895CF80180832115C8
:1055700031054105510521F0C22EE32FCA01E4CFC8
:10558000B801C7010E94FD29A196ECE00C94372ECA
:10559000A0E0B0E0EEECFAE20C941F2EEC016A0100
:1055A0007B012115310541F4E881F9810190F081F9
:1055B000E02D642F09951DC02A303105A9F477FF2D
:1055C00012C06DE20E943A2A8C0144275527BA0185
:1055D0004C195D096E097F092AE0CE010E948C2AD0
:1055E000800F911F06C02AE0B701A601CE010E94DC
:1055F0008C2ACDB7DEB7E8E00C943B2E9A01AB01C4
:10560000662757FD6095762F0E94C82A08950F934C
:105610001F93CF93DF93EC019A01AB01662757FDEF
:105620006095762F0E94C82A8C01CE010E94422AE2
:10563000800F911FDF91CF911F910F910895211538
:10564000310549F4DC01ED91FC910190F081E02DF0
:10565000642F099508950E948C2A08959A01462F77
:1056600050E060E070E00E941F2B08959A01AB01AA
:1056700060E070E00E941F2B08950F931F93CF935B
:10568000DF93EC010E941F2B8C01CE010E94422A65
:10569000800F911FDF91CF911F910F9108950F936C
:1056A0001F93CF93DF93EC019A01AB0160E070E0B0
:1056B0000E941F2B8C01CE010E94422A800F911F55
:1056C000DF91CF911F910F9108950F931F93CF9367
:1056D000DF93EC019A01462F50E060E070E00E94F9
:1056E0001F2B8C01CE010E94422A800F911FDF9157
:1056F000CF911F910F910895FC0124853585F90103
:10570000E05CFF4F80819181F901EE5BFF4F2081CA
:105710003181821B930B8F7399270895FC01848537
:105720009585FC01E05CFF4F40815181FC01EE5BFF
:10573000FF4F208131814217530741F00190F081E2
:10574000E02DE80FF91F808190E008958FEF9FEF23
:105750000895FC0184859585FC01E05CFF4F408144
:105760005181FC01EE5BFF4F2081318142175307CD
:1057700079F0A081B181A80FB91F8C91208131816E
:105780002F5F3F4F2F7333273183208390E008959D
:105790008FEF9FEF0895FC0181A1882329F0A48950
:1057A000B5898C9186FFFBCF11A20895CF93DF932B
:1057B000FC0126853785D901A05CBF4F8D919C9156
:1057C000119701968F739927E901CE5BDF4F4881CE
:1057D000598184179507D9F30D90BC91A02DA20F84
:1057E000B31F6C93A685B785A05CBF4F11969C93A1
:1057F0008E93A689B7892C9181E090E0078C02C036
:10580000880F991F0A94E2F7282B2C9381E081A33B
:105810000488F589E02D80818064808381E090E0B8
:10582000DF91CF91089508951F920F920FB60F92B6
:1058300011242F933F934F938F939F93EF93FF9355
:105840008091C00082FD1CC04091C60080918806F6
:105850009091890601968F73992720918A0630913D
:105860008B068217930771F0E0918806F091890604
:10587000E85BF94F4083909389068093880602C0C5
:105880008091C600FF91EF919F918F914F913F9131
:105890002F910F900FBE0F901F90189582EE95E0FC
:1058A0000E947C2B892B11F00E94132C08951F92CB
:1058B0000F920FB60F9211242F933F938F939F93C4
:1058C000EF93FF9320914406309145068091460660
:1058D000909147062817390731F48091C1008F7DD8
:1058E0008093C10014C0E0914606F0914706EC5F3A
:1058F000F94F2081809146069091470601968F735B
:10590000992790934706809346062093C600FF91FF
:10591000EF919F918F913F912F910F900FBE0F901C
:105920001F901895A0E0B0E0E8E9FCE20C941B2E73
:10593000FC011382128288EE93E0A0E0B0E0848341
:105940009583A683B7838CEB93E0918380837587DF
:10595000648757874687318B208B138B028BF58AA0
:10596000E48AD78AC68AB18EA08E938E828E8F8566
:10597000848F8889858F8989868F8A89878F8B898B
:1059800080A3ECE00C94372ECF92DF92EF92FF923F
:10599000CF93DF93EC016A017B01411581EE58073B
:1059A00061057105F9F0EC89FD8981E090E008A0BE
:1059B00002C0880F991F0A94E2F7808360E079E0C3
:1059C0008DE390E0A70196010E94D42D215031096A
:1059D000410951095695479537952795211580E13D
:1059E000380798F0EC89FD89108260E874E88EE150
:1059F00090E0A70196010E94D42D21503109410960
:105A000051095695479537952795E889F989308347
:105A1000EA89FB89208319A2EE89FF89408181E010
:105A200090E09C010C8C02C0220F331F0A94E2F715
:105A3000422B4083EE89FF8940819C010D8C02C07E
:105A4000220F331F0A94E2F7422B4083EE89FF892D
:105A500040819C010E8C02C0220F331F0A94E2F792
:105A6000422B4083EE89FF8920810F8C02C0880F72
:105A7000991F0A94E2F7809582238083DF91CF916A
:105A8000FF90EF90DF90CF9008958F929F92AF920A
:105A9000BF92CF92DF92EF92FF920F931F9381E01C
:105AA0008F9385E08F9387E08F9383E08F9384E0DB
:105AB0008F93E6EC8E2E912CF2ECAF2EB12CA1EC54
:105AC000CA2ED12CB0ECEB2EF12C04EC10E025EC1E
:105AD00030E044E056E068E476E082EE95E00E9433
:105AE000922C0F900F900F900F900F901F910F918D
:105AF000FF90EF90DF90CF90BF90AF909F908F90EE
:105B000008950E94C5280E942622CEE4DCE20E946D
:105B1000C4242097E1F30E944E2CF9CFA29FB0013C
:105B2000B39FC001A39F700D811D1124911DB29FD1
:105B3000700D811D1124911D08950E948E2DA59F29
:105B4000900DB49F900DA49F800D911D1124089578
:105B5000B7FF0C949D2D0E949D2D821B930B0895E1
:105B6000DB018F939F930E949D2DBF91AF91A29FC8
:105B7000800D911DA39F900DB29F900D112408954B
:105B800097FB072E16F4009407D077FD09D00E94EA
:105B9000522E07FC05D03EF4909581959F4F0895B5
:105BA000709561957F4F0895A1E21A2EAA1BBB1B29
:105BB000FD010DC0AA1FBB1FEE1FFF1FA217B307D9
:105BC000E407F50720F0A21BB30BE40BF50B661FEF
:105BD000771F881F991F1A9469F7609570958095B3
:105BE00090959B01AC01BD01CF010895052E97FB57
:105BF0001EF400940E940D2E57FD07D00E94D42D54
:105C000007FC03D04EF40C940D2E50954095309522
:105C100021953F4F4F4F5F4F089590958095709518
:105C200061957F4F8F4F9F4F08952F923F924F92D4
:105C30005F926F927F928F929F92AF92BF92CF921C
:105C4000DF92EF92FF920F931F93CF93DF93CDB725
:105C5000DEB7CA1BDB0B0FB6F894DEBF0FBECDBF9D
:105C600009942A88398848885F846E847D848C846E
:105C70009B84AA84B984C884DF80EE80FD800C8177
:105C80001B81AA81B981CE0FD11D0FB6F894DEBF5A
:105C90000FBECDBFED010895EE0FFF1F0590F491EB
:105CA000E02D0994AA1BBB1B51E107C0AA1FBB1F13
:105CB000A617B70710F0A61BB70B881F991F5A9598
:105CC000A9F780959095BC01CD0108958F929F9280
:105CD000AF92BF92CF92DF92EF92FF92CF93DF937A
:105CE000EC01688179818A819B816115710581054B
:105CF000910521F464E279ED8BE597E02DE133EF36
:105D000041E050E00E94F62D49015A019B01AC018F
:105D1000A7EAB1E40E949D2D6B017C01ACEEB4EFCB
:105D2000A50194010E94AB2DC60ED71EE81EF91ED8
:105D3000F7FE06C081E0C81AD108E10880E8F80A39
:105D4000C882D982EA82FB82C701B6019F77DF91C0
:105D5000CF91FF90EF90DF90CF90BF90AF909F904A
:105D60008F9008950E94662E089586E091E00E942B
:105D7000662E0895609306017093070180930801D1
:105D80009093090108952F923F925F926F927F92B4
:105D90008F929F92AF92BF92CF92DF92EF92FF923B
:105DA0000F931F93CF93DF938B01EA016115710568
:105DB00021F0DB018C9311969C93209739F09E0182
:105DC000225031092332310508F0D8C07C01670127
:105DD000BFEFCB1ADB0A5601F7016080862D90E0F9
:105DE0000E94F52F892B11F07601F1CFFDE26F12A1
:105DF0000AC0570182E0A80EB11CD70111966C9021
:105E0000772473940BC0BBE26B1207C05701E2E02A
:105E1000AE0EB11CD70111966C90712CCE018F7E05
:105E2000892B89F4B0E36B1237C0F50180818F7D37
:105E30008835D1F46180F2E0AF0EB11C872D82600D
:105E4000782EC0E1D0E0CA30D10551F1C031D10582
:105E500021F0C830D10599F409C0CC24CA94DC2CB7
:105E6000EC2CAFE0FA2E22C0209769F7C8E0D0E012
:105E7000CC24CA94DC2CEC2CFFE1FF2E17C06FEF72
:105E80007FEFCB019E01442737FD4095542F0E94A0
:105E9000D42D69017A010AC02097A9F6CAE0D0E0A2
:105EA000E9E9CE2EDC2CEC2CE9E1FE2EF50160E0D8
:105EB00020E030E0A9014E01AA2497FCA094BA2C5E
:105EC0001F0170ED572E560CA9E0A51570F48FEB4D
:105ED000860D8A3118F499EC592E06C08FE9860D8B
:105EE0008A3148F589EA582E560C852D90E08C179A
:105EF0009D070CF56F3FD9F0C216D306E406F506F0
:105F000098F0C501B4010E94B02D9B01AC01852D14
:105F100090E0A0E0B0E0280F391F4A1F5B1F281750
:105F200039074A075B0710F46FEF01C061E0319653
:105F3000D1016C90C5CF0115110551F0662311F008
:105F4000319703C071FE04C03297D801ED93FC93E2
:105F500070FE07C050954095309521953F4F4F4FAB
:105F60005F4F67FF10C082E290E090938D068093B0
:105F70008C066FEF7FEF8FEF9FEF07C060E070E060
:105F800080E090E002C0B901CA01DF91CF911F917A
:105F90000F91FF90EF90DF90CF90BF90AF909F90C8
:105FA0008F907F906F905F903F902F900895FC01AD
:105FB00088279927E89421912032E9F3293010F0BD
:105FC0002E30C8F32B3241F02D3239F4689404C0DE
:105FD0000E942930820F911D219120532A30C0F355
:105FE0001EF4909581959F4F0895911150C0803275
:105FF00019F089508550D0F7089548EC53E00E947D
:1060000002300895FA01A191B081009719F4109718
:10601000E1F0CD01DC01CD010D90002011F4C001B3
:1060200013C0FB012191222319F02015D9F7F3CFDA
:10603000FB012191201519F41E92119606C022230E
:10604000C1F70D900020A1F7D001FA01A193B08310
:1060500008957AE0979F902D879F802D910D1124B0
:106060000895F999FECF92BD81BDF89A992780B520
:106070000895262FF999FECF1FBA92BD81BD20BD8C
:106080000FB6F894FA9AF99A0FBE019608959927D7
:0860900088270895F894FFCF62
:1060980000008E06200001000000FF000200020040
:1060A80002000200020002000200020002000200D8
:1060B8000200020002000200020002802500000522
:1060C800400AA1204EA50020244EA52C2330C01242
:1060D80000001A400AA1204EA5001B1E27522C239F
:1060E800308025000005400AA1204EA50020244E3E
:1060F800A52C2330004B000006400AD0009D490023
:106108007B289D492C233000E1000005400A450109
:10611800D7DC03B81E0EBF00232E48E801008A40D2
:106128000A6001555502AD1E20000023C8015458CD
:106138002074696D656F75742100596573004E6F21
:10614800002C00386368004E2F41002C205B005D56
:106158002028002900486F70206368616E6E656CA6
:10616800200020402000456E746572696E672061CA
:1061780064617074697665206368616E6E656C2011
:1061880073656C656374696F6E2C207069636B69E5
:106198006E673A007363616E6E6572206D6F646539
:1061A800004E4F5420454E41424C45440053656EC5
:1061B80064696E672073657474696E677320746FA1
:1061C8002052580A00526573657474696E672073AB
:1061D800657474696E6773206F6E2052580A0041A7
:1061E800626F727465642065646974730A00696E0D
:1061F80076616C69642073656C656374696F6E00A1
:106208000D0A496E76616C696420696E7075742038
:106218002D206469736361726465642107005365A6
:106228007474696E677320736176656420746F2077
:10623800454550524F4D0A00526576657274656443
:106248002073657474696E67732066726F6D20457C
:106258004550524F4D0A004C6F6164656420666179
:1062680063746F72792064656661756C74730A0073
:106278004B657920616E64206368616E6E656C732E
:106288002072616E646F6D697A65640A004F70658B
:106298006E4C52536E67205458207374617274693F
:1062A8006E672000206F6E20485720006D6F647560
:1062B8006C65206C6F636B65643F00342B34003869
:1062C80000382B340031320031322B3400313600A3
:1062D80050504D0052535349005344410053434CCE
:1062E80000525844005458440041494E004C42451D
:1062F80045500053504B54524D0053425553005390
:10630800554D44004C4C494E440000070B0C1011ED
:106318001500B7012B032F033103350338033D0361
:10632800B7014003440349034D035103550359037F
:106338005D0363036A036F0374038D028D028D028C
:106348008D02160A1322312900000000D62BDB2902
:086358007C2BA92B8E2BCB2B13
:107E00000F92CDB7DEB7112484B714BE81FFF1D035
:107E100082E08093C00088E18093C10086E0809377
:107E2000C20080E18093C4008EE0CDD088249924E4
:107E3000CC24C394F5E0DF2EE1E1EE2E73E0F72EC3
:107E4000B6D0082F813479F4B2D08983C2D0898129
:107E5000823811F481E005C0813811F485E001C059
:107E600083E09ED09AC0823411F484E103C085344B
:107E700019F485E0B6D091C0853561F498D0082F0B
:107E800010E095D090E0982E8824802A912A880CC2
:107E9000991C82C0863521F484E0A3D080E0E1CF34
:107EA000843609F04CC083D082D0A82E80D0B82E62
:107EB00000E011E07CD0F80181938F01AE16D1F77C
:107EC00088D0FB2DF53489F4E0E0F1E00BC0F9999E
:107ED000FECF92BC81BC0894811C911C819180BD15
:107EE000FA9AF99AEA1598F358C08B2D863409F05E
:107EF00054C0F401F7BEE89507B600FCFDCFF401CD
:107F0000A0E0B1E02C9130E011968C91119790E0B7
:107F1000982F8827822B932B12960C01C7BEE895C9
:107F20001124329681E0A038B80761F7F401D7BE7A
:107F3000E89507B600FCFDCFE7BEE8952EC0843774
:107F4000F1F435D034D0182F32D0B82E42D0FB2DDA
:107F5000F63421F4F40105914F010CC0FB2DF534EA
:107F600049F4F999FECF92BC81BC0894811C911C04
:107F7000F89A00B5802F14D0115049F70EC08537FC
:107F800039F427D08EE10CD085E90AD08FE069CF93
:107F9000813511F488E017D01CD080E101D050CF9A
:107FA0009091C00095FFFCCF8093C600089580910A
:107FB000C00087FFFCCF8091C00084FD01C0A89560
:107FC0008091C6000895E0E6F0E098E19083808318
:107FD0000895EDDF803219F088E0F5DFFFCF84E10E
:107FE000DFCF1F93182FE3DF1150E9F7F2DF1F9166
:0E7FF0000895282E80E0E7DFEE27FF27099492
:027FFE0001057B
:0400000300007E007B
:00000001FF
